:100000008A01F628820730343134323433343434C0
:100010003534363437343834393441344234433467
:10002000443445344634981C1728181218168C1E70
:100030002A28000000001A08A2002208383C031CED
:100040002A2831302202031C2A2830302202A30041
:10005000A20108006D302206031D31280830A300DC
:1000600008006830220603196627A2011328FF3012
:10007000A100A10B392808009900000000000C1E07
:100080003F280800270E0F3902203C2027080F398F
:1000900002203C20260E0F3902203C2026080F3972
:1000A00002203C2020303C20290E0F3902203C2029
:1000B00029080F3902203C20280E0F3902203C204D
:1000C00028080F3902203C202303031908002030A0
:1000D0003C200800AC09AC0A0319AD03AD092C089B
:1000E000AA070318AB0A2D08AB0708002A08A607C1
:1000F0000318A70A2B08A70708008F018E010530F7
:1001000097000C1110140C1017148F1ADA280C1DFC
:1001100085280C112E30840015088000840A1608EA
:1001200080000A30A00017100C18DA280C1D942843
:100130000C11840A15088000840A16088000171420
:100140000C18DA280C1DA0280C11840A1508800050
:10015000840A16088000A00B9328A601A701A80115
:10016000A9010A30A0002E3084008403840A00080C
:10017000AC00840A0008AD00840A0008AA00840AC2
:100180000008AB006A207620A00BB628840A00087D
:10019000AA00840A0008AB002E3084000008AC00DE
:1001A000840A0008AD006A202A08A8002B08A900CC
:1001B0004220080097011010FF30A600A700A800F9
:1001C000A900422008000130A400A50124088600EF
:1001D0002508850037207D202408A407A50AA30B45
:1001E000E6280D303C200A303C2008008316803081
:1001F00081008312860185018316383085008601CF
:10020000FF3087001530990098161815831298173B
:0E021000181690019701A2011320E3200C297B
:0809F80021088A002008820793
:100A00000D340A342034203420342034203420346F
:100A10002034533420344D34203454342034413481
:100A200020345334203438342034203420345434A7
:100A30002034453420344D3420345034203445346F
:100A4000203452342034413420345434203455344A
:100A500020345234203445340D340A3420342034C8
:100A6000203420342034203420344D342034453494
:100A7000203441342034533420345534203452341B
:100A80002034453420344D342034453420344E3421
:100A90002034543420342034203453342034593416
:100AA00020345334203454342034453420344D34ED
:100AB0000D340A34203420342034203420342034BF
:100AC0002034203420342034203420342034563450
:100AD00065347234733469346F346E342034313495
:100AE0002E34303420342F342034303431342E340A
:100AF000303434342E3432343034303432340D34F3
:100B00000A340D340A342034203420342034203484
:100B10006D3420342D343E34203449346E34663400
:100B200069346E3469347434653420346D3465341A
:100B3000613473347534723465346D3465346E34B5
:100B4000743420346334793463346C3465340D3454
:100B50000A342034203420342034203431342034FA
:100B60002D343E3420344634693472347334743452
:100B70002034733465346E3473346F3472342C34EF
:100B80002034733469346E3467346C346534203403
:100B90006D346534613473347534723465346D3456
:100BA00065346E3474340D340A34203420342034E7
:100BB00020342034323420342D343E342034463432
:100BC00069347234733474342034743477346F3449
:100BD0002034733465346E3473346F347234733448
:100BE0002C342034733469346E3467346C34653497
:100BF00020346D3465346134733475347234653443
:100C00006D3465346E3474340D340A342034203439
:100C1000203420342034333420342D343E342034F6
:100C20004634693472347334743420347434683420
:100C30007234653465342034733465346E347334FF
:100C40006F34723473342C342034733469346E341A
:100C500067346C34653420346D34653461347334F6
:100C60007534723465346D3465346E3474340D34D7
:100C70000A342034203420342034203434342034D6
:100C80002D343E3420344634693472347334743431
:100C9000203466346F3475347234203473346534E0
:100CA0006E3473346F34723473342C3420347334B0
:100CB00069346E3467346C34653420346D34653493
:100CC000613473347534723465346D3465346E3424
:100CD00074340D340A342034203420342034203449
:100CE000353420342D343E34203446346934723463
:100CF0007334743420346634693476346534203483
:100D0000733465346E3473346F34723473342C340A
:100D10002034733469346E3467346C346534203471
:100D20006D346534613473347534723465346D34C4
:100D300065346E3474340D340A3420342034203455
:100D400020342034363420342D343E34203446349C
:100D500069347234733474342034733469347834BD
:100D60002034733465346E3473346F3472347334B6
:100D70002C342034733469346E3467346C34653405
:100D800020346D34653461347334753472346534B1
:100D90006D3465346E3474340D340A3420342034A8
:100DA000203420342034373420342D343E34203461
:100DB0004634693472347334743420347334653493
:100DC000763465346E342034733465346E34733461
:100DD0006F34723473342C342034733469346E3489
:100DE00067346C34653420346D3465346134733465
:100DF0007534723465346D3465346E3474340D3446
:100E00000A34203420342034203420343834203440
:100E10002D343E342034463469347234733474349F
:100E2000203465346934673468347434203473345E
:100E300065346E3473346F34723473342C3420342C
:100E4000733469346E3467346C34653420346D34F3
:100E50006534613473347534723465346D3465349B
:100E60006E3474340D340A34203420342034203469
:100E70002034733420342D343E34203453347434CD
:100E80006F3470340D340A340D340A342034203475
:100E900020342034203450346C346534613473345D
:100EA000653420344D3461346B346534203461341E
:100EB0002034433468346F34693463346534203407
:100EC0003A340D340A340D340A342A34A000053083
:100ED000A100FC24A2002A3022060319762F220842
:100EE0003C200130A0070318A10A692F00308A00B6
:020EF0000800F8
:02400E00020F9F
:00000001FF
